:100000001AC091C0A7C030C02FC02EC02DC02CC0B8
:100010002BC02AC029C028C027C027C025C024C0A3
:1000200023C022C021C0E1C0F0C00BC11FC12DC13F
:1000300048C162C17BC111241FBECFEDCDBF10E00E
:10004000A0E6B0E0E8E6F3E002C005900D92A2362B
:10005000B107D9F710E0A2E6B0E001C01D92A836C2
:10006000B107E1F785D07EC1CBCF1F920F920FB6BB
:100070000F9211248F939F93AF93BF93809164004D
:1000800090916500A0916600B09167000196A11D56
:10009000B11D8093640090936500A0936600B093B7
:1000A00067008091640090916500A0916600B09116
:1000B0006700892B8A2B8B2B59F48FEF9FEFDC0184
:1000C0008093640090936500A0936600B0936700EE
:1000D000809163008823F1F080916000909161002D
:1000E00001969093610080936000809160009091F0
:1000F0006100892B31F48FEF9FEF90936100809323
:1001000060008091600090916100069710F4959ACC
:1001100001C09598BF91AF919F918F910F900FBEA5
:100120000F901F9018951F920F920FB60F921124E7
:100130008F9380916300833021F08091630082303F
:1001400019F481E0809363008F910F900FBE0F90A0
:100150001F9018951F920F920FB60F9211241092B4
:100160006100109260000F900FBE0F901F901895C5
:100170008E9A8D9A8C9A969A959A949AC09AC19AC8
:10018000B99AC29ABA9AC39ABB9ABC9A82E080BFC3
:1001900083E083BF8CE786BF81E089BF85B782603B
:1001A00085BF8BB780648BBF85B7846085BF8BB7F5
:1001B00080688BBF78941092640010926500109252
:1001C0006600109267001092630081E097E026E0DD
:1001D00035E044E053E062E0E0916300F0E0E830B5
:1001E000F105D0F7ED5EFF4F0994C0906400D09008
:1001F0006500E0906600F090670078E8C71673E14C
:10020000D706E104F10440F3AAC0C19AC29AC39A86
:10021000969AC4989498E0916000F09161003697A6
:10022000D8F6B099D9CFC49A949A969860936300FF
:1002300010926400109265001092660010926700A0
:10024000CBCFC0906400D0906500E0906600F09045
:1002500067007EE4C7167DE0D706E104F10408F4E8
:10026000BBCFC498C29850936300B6CFB09BB4CFB5
:10027000C198969A109264001092650010926600E0
:100280001092670040936300A7CFC0906400D090A5
:100290006500E0906600F090670079E4C71673E0AF
:1002A000D706E104F10408F497CFC39810926400D4
:1002B0001092650010926600109267003093630000
:1002C0008BCFC0906400D0906500E0906600F09005
:1002D000670075EDC716D104E104F10408F47CCF82
:1002E000C29A1092640010926500109266001092FB
:1002F00067002093630070CFC0906400D0906500C9
:10030000E0906600F090670077E3C71671E0D706CB
:10031000E104F10458F0C19A109264001092650053
:10032000109266001092670090936300C090640082
:10033000D0906500E0906600F090670071E5C71608
:1003400073E0D706E104F10408F446CFC39A109293
:10035000640010926500109266001092670080930E
:0803600063003ACFF894FFCFCF
:0203680006008D
:00000001FF
